Microsoft (R) Macro Assembler Version 5.10                  2/14/25 23:44:14
CHKPRMT - Procedures called from chkdsk which prompt			;an00Page     1-1


				TITLE	CHKPRMT - Procedures called from chkdsk
				 which prompt			;an000;bgb
				page	,132					;				;an000;bgb
														;an000;bgb
					.list									;an000;bgb
														;an000;bgb
														;an000;bgb
 0000				CONST	SEGMENT PUBLIC PARA 'DATA'						;an000;bgb
					EXTRN	YES_BYTE:BYTE,NO_BYTE:BYTE					;an000;bgb
					EXTRN	YN_ARG:WORD							;an000;bgb
					EXTRN	HECODE:byte,CONBUF:byte 					;an000;bgb
 0000				CONST	ENDS									;an000;bgb
														;an000;bgb
														;an000;bgb
 0000				CODE	SEGMENT PUBLIC PARA 'CODE'						;an000;bgb
				ASSUME	CS:DG,DS:DG,ES:DG,SS:DG 						;an000;bgb
					EXTRN	PRINTF_CRLF:NEAR,DOCRLF:NEAR					;an000;bgb
														;an000;bgb
					pathlabl chkprmt							;an000;bgb
				;*****************************************************************************	;an000;bgb
				;Routine name:PromptYN								;an000;bgb
				;*****************************************************************************	;an000;bgb
				;										;an000;bgb
				;description: Validate that input is valid Y/N for the country dependent info	;an000;bgb
				;	     Return Z flag if 'Y' entered					;an000;bgb
				;Called Procedures: Message (macro)						;an000;bgb
				;		    User_String 						;an000;bgb
				;										;an000;bgb
				;Change History: Created	5/10/87 	MT				;an000;bgb
				;										;an000;bgb
				;Input: DX = offset to message							;an000;bgb
				;										;an000;bgb
				;Output: Z flag if 'Y' entered							;an000;bgb
				;										;an000;bgb
				;Psuedocode									;an000;bgb
				;----------									;an000;bgb
				;										;an000;bgb
				;	DO									;an000;bgb
				;	   Display prompt and input character					;an000;bgb
				;	   IF got character							;an000;bgb
				;	      Check for country dependent Y/N (INT 21h, AX=6523h Get Ext Country;an000;bgb)
				;	      IF NC (Yes or No) 						;an000;bgb
				;		 Set Z if Yes, NZ if No 					;an000;bgb
				;	      ENDIF								;an000;bgb
				;	   ELSE  (nothing entered)						;an000;bgb
				;	      stc								;an000;bgb
				;	   ENDIF								;an000;bgb
				;	ENDDO NC								;an000;bgb
				;	ret									;an000;bgb
				;*****************************************************************************	;an000;bgb
				Procedure PromptYN				;				;an000;bgb;AN000;
			     1							; 
			     1	Public	PromptYN				;				;AN000; 
 0000                        1	PromptYN    proc				;				;AN000; 
Microsoft (R) Macro Assembler Version 5.10                  2/14/25 23:44:14
CHKPRMT - Procedures called from chkdsk which prompt			;an00Page     1-2
system call definitions                                     

 0000  56				push	si				;Save reg			;an000;bgb
				;	$DO					;				;an000;bgb;AC000;
 0001				$$DO1:
 0001  E8 0000 E			   Call    Display_Interface		;Display the message		;an000;bgb;AC000;
 0004  BA 0000 E			   MOV	   DX,OFFSET DG:CONBUF		;Point at input buffer		;an000;bgb
					   DOS_Call Std_Con_String_Input	;Get input			;an000;bgb;AC000;
			     1							; 
 0007  B4 0A                 1		mov	ah,Std_Con_String_Input			;				;AN000; 
 0009  CD 21                 1		int	21h				;				;AN000; 
			     1							; 
 000B  E8 0000 E			   CALL    DOCRLF			;				;an000;bgb
 000E  BE 0002 E			   MOV	   SI,OFFSET DG:CONBUF+2	;Point at contents of buffer	;an000;bgb
 0011  80 7C FF 00			   CMP	   BYTE PTR [SI-1],0		;Was there input?		;an000;bgb
				;	   $IF	   NE				;Yep				;an000;bgb;AC000;
 0015  74 10				   JE $$IF2
 0017  B0 23				      mov     al,23h			;See if it is Y/N		;an000;bgb;AN000;
 0019  8A 14				      mov     dl,[si]			;Get character			;an000;bgb;AN000;
					      DOS_Call GetExtCntry		;Get country info call		;an000;bgb;AN000;
			     1							; 
 001B  B4 65                 1		mov	ah,GetExtCntry			;				;AN000; 
 001D  CD 21                 1		int	21h				;				;AN000; 
			     1							; 
				;	      $IF     NC			;Yes or No entered		;an000;bgb;AN000;
 001F  72 04				      JC $$IF3
 0021  3D 0001					 cmp	 ax,Yes_Found		;Set Z if Yes, NZ if No 	;an000;bgb;AN000;
 0024  F8					 clc				;CY=0 means Y/N found		;an000;bgb
				;	      $ENDIF				;CY set if neither		;an000;bgb;AN000;
 0025				$$IF3:
				;	   $ELSE				;No characters input		;an000;bgb
 0025  EB 01				   JMP SHORT $$EN2
 0027				$$IF2:
 0027  F9				      stc				;CY means not Y/N		;an000;bgb
				;	   $ENDIF				;				;an000;bgb
 0028				$$EN2:
				;	$ENDDO	NC				;				;an000;bgb;AN000;
 0028  72 D7				JC $$DO1
 002A  5E				pop	si				;				;an000;bgb
 002B  C3				ret					;				;an000;bgb
 002C				PromptYN endp					;				;an000;bgb;AN000;
					pathlabl chkprmt							;an000;bgb
														;an000;bgb
 002C				CODE	ENDS									;an000;bgb
					END									;an000;bgb

Microsoft (R) Macro Assembler Version 5.10                  2/14/25 23:44:14
CHKPRMT - Procedures called from chkdsk which prompt			;an00Symbols-1


Macros:

		N a m e			Lines

BREAK  . . . . . . . . . . . . .  	   2
DOS_CALL . . . . . . . . . . . .  	   4
EXTENDED_MESSAGE . . . . . . . .  	   8
MESSAGE  . . . . . . . . . . . .  	   4
PARSE_MESSAGE  . . . . . . . . .  	   8
PATHLABL . . . . . . . . . . . .  	  10
POPFF  . . . . . . . . . . . . .  	   6
PROCEDURE  . . . . . . . . . . .  	   3
SET_DATA_SEGMENT . . . . . . . .  	   9

Structures and Records:

                N a m e                 Width   # fields
                                        Shift   Width   Mask    Initial

A_DEVICEPARAMETERS . . . . . . .  	0026	0012
  SPECIALFUNCTIONS . . . . . . .  	0000
  DEVICETYPE . . . . . . . . . .  	0001
  DEVICEATTRIBUTES . . . . . . .  	0002
  NUMBEROFCYLINDERS  . . . . . .  	0004
  MEDIATYPE  . . . . . . . . . .  	0006
  BYTEPERSECTOR  . . . . . . . .  	0007
  SECTORSPERCLUSTER  . . . . . .  	0009
  RESERVEDSECTORS  . . . . . . .  	000A
  NUMBEROFFATS . . . . . . . . .  	000C
  ROOTENTRIES  . . . . . . . . .  	000D
  TOTALSECTORS . . . . . . . . .  	000F
  MEDIADESCRIPTOR  . . . . . . .  	0011
  SECTORSPERFAT  . . . . . . . .  	0012
  SECTORSPERTRACK  . . . . . . .  	0014
  HEADS  . . . . . . . . . . . .  	0016
  HIDDENSECTORS  . . . . . . . .  	0018
  EXT_TOTAL_SECTORS  . . . . . .  	001C
  RESERVEDAREA . . . . . . . . .  	0020
DIRENT . . . . . . . . . . . . .  	0028	000C
  DIRNAM . . . . . . . . . . . .  	0008
  DIRATT . . . . . . . . . . . .  	0013
  DIRCP  . . . . . . . . . . . .  	0014
  DIR_XA . . . . . . . . . . . .  	0016
  DIRATT2  . . . . . . . . . . .  	0018
  DIRRES . . . . . . . . . . . .  	0019
  DIRTIM . . . . . . . . . . . .  	001E
  DIRDAT . . . . . . . . . . . .  	0020
  DIRCLUS  . . . . . . . . . . .  	0022
  DIRESIZ  . . . . . . . . . . .  	0024
RELATIVE_SECTOR_BUFFER . . . . .  	000A	0005
  START_SECTOR_LOW . . . . . . .  	0000
  START_SECTOR_HIGH  . . . . . .  	0002
  NUMBER_SECTORS . . . . . . . .  	0004
  BUFFER_OFFSET  . . . . . . . .  	0006
Microsoft (R) Macro Assembler Version 5.10                  2/14/25 23:44:14
CHKPRMT - Procedures called from chkdsk which prompt			;an00Symbols-2


  BUFFER_SEGMENT . . . . . . . .  	0008
SUBLIST_STRUC  . . . . . . . . .  	000B	0009
  SUBLIST_SIZE . . . . . . . . .  	0000
  SUBLIST_RSV  . . . . . . . . .  	0001
  SUBLIST_OFFSET . . . . . . . .  	0002
  SUBLIST_SEGMENT  . . . . . . .  	0004
  SUBLIST_NUMBER . . . . . . . .  	0006
  SUBLIST_TYPE . . . . . . . . .  	0007
  SUBLIST_MAX  . . . . . . . . .  	0008
  SUBLIST_MIN  . . . . . . . . .  	0009
  SUBLIST_CHAR . . . . . . . . .  	000A
XAL  . . . . . . . . . . . . . .  	0200	0005
  XAL_TSIZE  . . . . . . . . . .  	0000
  XAL_TCOUNT . . . . . . . . . .  	0002
  XAL_LSIZE  . . . . . . . . . .  	0004
  XAL_LCOUNT . . . . . . . . . .  	0006
  XAL_DATA . . . . . . . . . . .  	0008

Segments and Groups:

                N a m e         	Length	 Align	Combine Class

DG . . . . . . . . . . . . . . .  	GROUP
  DATA . . . . . . . . . . . . .  	0000	PARA	PUBLIC	'DATA'
  CONST  . . . . . . . . . . . .  	0000	PARA	PUBLIC	'DATA'
  CODE . . . . . . . . . . . . .  	002C	PARA	PUBLIC	'CODE'
  CSTACK . . . . . . . . . . . .  	0000	PARA	STACK	'STACK'
  LASTSEG  . . . . . . . . . . .  	0000	PARA	PUBLIC	'LAST'
PSP  . . . . . . . . . . . . . .  	0000	PARA	PUBLIC	'DUMMY'

Symbols:            

                N a m e         	Type	 Value	 Attr

ABORT  . . . . . . . . . . . . .  	NUMBER	0000	
ALLOC  . . . . . . . . . . . . .  	NUMBER	0048	
ALLOCOPER  . . . . . . . . . . .  	NUMBER	0058	
APPEND_OFF . . . . . . . . . . .  	NUMBER	0000	
APPEND_ON  . . . . . . . . . . .  	NUMBER	0001	
APPEND_X . . . . . . . . . . . .  	NUMBER	B706	
APPEND_X_SET . . . . . . . . . .  	NUMBER	0001	
ASCIIZ_END . . . . . . . . . . .  	NUMBER	0000	
ASSIGNOPER . . . . . . . . . . .  	NUMBER	005F	
ASSIGN_CHECK . . . . . . . . . .  	NUMBER	8000	

BAD_EXIT . . . . . . . . . . . .  	NUMBER	00FF	
BIG_FAT_THRESHOLD  . . . . . . .  	NUMBER	0FF6	
BLANK  . . . . . . . . . . . . .  	NUMBER	0020	

CHAR_OPER  . . . . . . . . . . .  	NUMBER	0037	
CHDIR  . . . . . . . . . . . . .  	NUMBER	003B	
CHK_ERROR  . . . . . . . . . . .  	NUMBER	0001	
CHMOD  . . . . . . . . . . . . .  	NUMBER	0043	
Microsoft (R) Macro Assembler Version 5.10                  2/14/25 23:44:14
CHKPRMT - Procedures called from chkdsk which prompt			;an00Symbols-3


CLOSE  . . . . . . . . . . . . .  	NUMBER	003E	
COMMIT . . . . . . . . . . . . .  	NUMBER	0068	
CONBUF . . . . . . . . . . . . .  	V BYTE	0000	CONST	External
CREAT  . . . . . . . . . . . . .  	NUMBER	003C	
CREATENEWFILE  . . . . . . . . .  	NUMBER	005B	
CREATETEMPFILE . . . . . . . . .  	NUMBER	005A	
CREATE_PROCESS_DATA_BLOCK  . . .  	NUMBER	0026	
CRITICAL_ERROR_FAIL  . . . . . .  	NUMBER	0003	
CURRENT_DIR  . . . . . . . . . .  	NUMBER	0047	

DAY_MASK . . . . . . . . . . . .  	NUMBER	001F	
DEALLOC  . . . . . . . . . . . .  	NUMBER	0049	
DIR_ATTRIBUTE  . . . . . . . . .  	NUMBER	0010	
DIR_ENTRIES_PER_SECTOR . . . . .  	NUMBER	0010	
DIR_SEARCH_FIRST . . . . . . . .  	NUMBER	0011	
DIR_SEARCH_NEXT  . . . . . . . .  	NUMBER	0012	
DISK_ERROR . . . . . . . . . . .  	NUMBER	0080	
DISK_RESET . . . . . . . . . . .  	NUMBER	000D	
Display_Interface  . . . . . . .  	L NEAR	0000		External
DOCRLF . . . . . . . . . . . . .  	L NEAR	0000	CODE	External
DO_INCLUDE . . . . . . . . . . .  	NUMBER	0001	
DRIVE_NOT_READY  . . . . . . . .  	NUMBER	0002	
DRVCHAR  . . . . . . . . . . . .  	NUMBER	003A	
DUP_PDB  . . . . . . . . . . . .  	NUMBER	0055	

ECS_CALL . . . . . . . . . . . .  	NUMBER	0063	
ENTSIZ . . . . . . . . . . . . .  	NUMBER	0028	
EXEC . . . . . . . . . . . . . .  	NUMBER	004B	
EXIT . . . . . . . . . . . . . .  	NUMBER	004C	
EXTHANDLE  . . . . . . . . . . .  	NUMBER	0067	
EXTOPEN  . . . . . . . . . . . .  	NUMBER	006C	

FALSE  . . . . . . . . . . . . .  	NUMBER	0000	
FCB  . . . . . . . . . . . . . .  	NUMBER	005C	
FCB_CLOSE  . . . . . . . . . . .  	NUMBER	0010	
FCB_CREATE . . . . . . . . . . .  	NUMBER	0016	
FCB_DELETE . . . . . . . . . . .  	NUMBER	0013	
FCB_OPEN . . . . . . . . . . . .  	NUMBER	000F	
FCB_RANDOM_READ  . . . . . . . .  	NUMBER	0021	
FCB_RANDOM_READ_BLOCK  . . . . .  	NUMBER	0027	
FCB_RANDOM_WRITE . . . . . . . .  	NUMBER	0022	
FCB_RANDOM_WRITE_BLOCK . . . . .  	NUMBER	0028	
FCB_RENAME . . . . . . . . . . .  	NUMBER	0017	
FCB_SEQ_READ . . . . . . . . . .  	NUMBER	0014	
FCB_SEQ_WRITE  . . . . . . . . .  	NUMBER	0015	
FILE_TIMES . . . . . . . . . . .  	NUMBER	0057	
FIND_FIRST . . . . . . . . . . .  	NUMBER	004E	
FIND_NEXT  . . . . . . . . . . .  	NUMBER	004F	
FOUND_NO . . . . . . . . . . . .  	NUMBER	0000	
FOUND_YES  . . . . . . . . . . .  	NUMBER	0001	

GETCURRENTPSP  . . . . . . . . .  	NUMBER	0062	
GETEXTCNTRY  . . . . . . . . . .  	NUMBER	0065	
GETEXTENDEDERROR . . . . . . . .  	NUMBER	0059	
Microsoft (R) Macro Assembler Version 5.10                  2/14/25 23:44:14
CHKPRMT - Procedures called from chkdsk which prompt			;an00Symbols-4


GETSETCDPG . . . . . . . . . . .  	NUMBER	0066	
GETSETMEDIAID  . . . . . . . . .  	NUMBER	0069	
GET_CURRENT_PDB  . . . . . . . .  	NUMBER	0051	
GET_DATE . . . . . . . . . . . .  	NUMBER	002A	
GET_DEFAULT_DPB  . . . . . . . .  	NUMBER	001F	
GET_DEFAULT_DRIVE  . . . . . . .  	NUMBER	0019	
GET_DMA  . . . . . . . . . . . .  	NUMBER	002F	
GET_DPB  . . . . . . . . . . . .  	NUMBER	0032	
GET_DRIVE_FREESPACE  . . . . . .  	NUMBER	0036	
GET_FCB_FILE_LENGTH  . . . . . .  	NUMBER	0023	
GET_FCB_POSITION . . . . . . . .  	NUMBER	0024	
GET_INDOS_FLAG . . . . . . . . .  	NUMBER	0034	
GET_INTERRUPT_VECTOR . . . . . .  	NUMBER	0035	
GET_IN_VARS  . . . . . . . . . .  	NUMBER	0052	
GET_TIME . . . . . . . . . . . .  	NUMBER	002C	
GET_VERIFY_ON_WRITE  . . . . . .  	NUMBER	0054	
GET_VERSION  . . . . . . . . . .  	NUMBER	0030	

HEAD_MASK  . . . . . . . . . . .  	NUMBER	007F	
HECODE . . . . . . . . . . . . .  	V BYTE	0000	CONST	External
HIDDN  . . . . . . . . . . . . .  	NUMBER	0002	
HONGEUL  . . . . . . . . . . . .  	NUMBER	0063	
HOUR_MASK  . . . . . . . . . . .  	NUMBER	F800	

IFS_IOCTL  . . . . . . . . . . .  	NUMBER	006B	
INTERNATIONAL  . . . . . . . . .  	NUMBER	0038	
IOCTL  . . . . . . . . . . . . .  	NUMBER	0044	
ISDIR  . . . . . . . . . . . . .  	NUMBER	0010	

KEEP_PROCESS . . . . . . . . . .  	NUMBER	0031	

LBL_CHKPRMT  . . . . . . . . . .  	NUMBER	0001	
LOCKOPER . . . . . . . . . . . .  	NUMBER	005C	
LSEEK  . . . . . . . . . . . . .  	NUMBER	0042	

MINUTE_MASK  . . . . . . . . . .  	NUMBER	07E0	
MKDIR  . . . . . . . . . . . . .  	NUMBER	0039	
MONTH_MASK . . . . . . . . . . .  	NUMBER	01E0	
MULTIPLEX  . . . . . . . . . . .  	NUMBER	002F	

NET_CHECK  . . . . . . . . . . .  	NUMBER	1200	
NO . . . . . . . . . . . . . . .  	NUMBER	0000	
NOT_INCLUDE  . . . . . . . . . .  	NUMBER	0000	
NO_BYTE  . . . . . . . . . . . .  	V BYTE	0000	CONST	External
NO_ENTRY . . . . . . . . . . . .  	NUMBER	0000	
NO_ERROR . . . . . . . . . . . .  	NUMBER	0000	
NO_EXT_ATTRIB  . . . . . . . . .  	NUMBER	0000	
NO_FOUND . . . . . . . . . . . .  	NUMBER	0000	

OEM_C1 . . . . . . . . . . . . .  	NUMBER	00F9	
OEM_C2 . . . . . . . . . . . . .  	NUMBER	00FA	
OEM_C3 . . . . . . . . . . . . .  	NUMBER	00FB	
OEM_C4 . . . . . . . . . . . . .  	NUMBER	00FC	
OEM_C5 . . . . . . . . . . . . .  	NUMBER	00FD	
Microsoft (R) Macro Assembler Version 5.10                  2/14/25 23:44:14
CHKPRMT - Procedures called from chkdsk which prompt			;an00Symbols-5


OEM_C6 . . . . . . . . . . . . .  	NUMBER	00FE	
OEM_C7 . . . . . . . . . . . . .  	NUMBER	00FF	
OFF  . . . . . . . . . . . . . .  	NUMBER	0000	
ON . . . . . . . . . . . . . . .  	NUMBER	0001	
OPEN . . . . . . . . . . . . . .  	NUMBER	003D	

PARSE_FILE_DESCRIPTOR  . . . . .  	NUMBER	0029	
PATHPARSE  . . . . . . . . . . .  	NUMBER	0061	
PRINTF_CRLF  . . . . . . . . . .  	L NEAR	0000	CODE	External
PromptYN . . . . . . . . . . . .  	N PROC	0000	CODE	Global	Length = 002C

RAW_CON_INPUT  . . . . . . . . .  	NUMBER	0007	
RAW_CON_IO . . . . . . . . . . .  	NUMBER	0006	
RDONLY . . . . . . . . . . . . .  	NUMBER	0001	
READ . . . . . . . . . . . . . .  	NUMBER	003F	
RENAME . . . . . . . . . . . . .  	NUMBER	0056	
RMDIR  . . . . . . . . . . . . .  	NUMBER	003A	

SERVERCALL . . . . . . . . . . .  	NUMBER	005D	
SETBLOCK . . . . . . . . . . . .  	NUMBER	004A	
SETDPB . . . . . . . . . . . . .  	NUMBER	0053	
SET_APPEND_X . . . . . . . . . .  	NUMBER	B707	
SET_CTRL_C_TRAPPING  . . . . . .  	NUMBER	0033	
SET_CURRENT_PDB  . . . . . . . .  	NUMBER	0050	
SET_DATE . . . . . . . . . . . .  	NUMBER	002B	
SET_DEFAULT_DRIVE  . . . . . . .  	NUMBER	000E	
SET_DMA  . . . . . . . . . . . .  	NUMBER	001A	
SET_INTERRUPT_VECTOR . . . . . .  	NUMBER	0025	
SET_OEM_HANDLER  . . . . . . . .  	NUMBER	00F8	
SET_PRINTER_FLAG . . . . . . . .  	NUMBER	0064	
SET_TIME . . . . . . . . . . . .  	NUMBER	002D	
SET_VERIFY_ON_WRITE  . . . . . .  	NUMBER	002E	
STDERR . . . . . . . . . . . . .  	NUMBER	0002	
STD_AUX_INPUT  . . . . . . . . .  	NUMBER	0003	
STD_AUX_OUTPUT . . . . . . . . .  	NUMBER	0004	
STD_CON_INPUT  . . . . . . . . .  	NUMBER	0001	
STD_CON_INPUT_FLUSH  . . . . . .  	NUMBER	000C	
STD_CON_INPUT_NO_ECHO  . . . . .  	NUMBER	0008	
STD_CON_INPUT_STATUS . . . . . .  	NUMBER	000B	
STD_CON_OUTPUT . . . . . . . . .  	NUMBER	0002	
STD_CON_STRING_INPUT . . . . . .  	NUMBER	000A	
STD_CON_STRING_OUTPUT  . . . . .  	NUMBER	0009	
STD_PRINTER_OUTPUT . . . . . . .  	NUMBER	0005	
STRING_DONE  . . . . . . . . . .  	NUMBER	0000	
SYSTM  . . . . . . . . . . . . .  	NUMBER	0004	

THISENT  . . . . . . . . . . . .  	NUMBER	0014	
TRUE . . . . . . . . . . . . . .  	NUMBER	FFFF	

UNLINK . . . . . . . . . . . . .  	NUMBER	0041	
USEROPER . . . . . . . . . . . .  	NUMBER	005E	

VOLIDA . . . . . . . . . . . . .  	NUMBER	0008	
VOL_ATTRIBUTE  . . . . . . . . .  	NUMBER	0008	
Microsoft (R) Macro Assembler Version 5.10                  2/14/25 23:44:14
CHKPRMT - Procedures called from chkdsk which prompt			;an00Symbols-6



WAITPROCESS  . . . . . . . . . .  	NUMBER	004D	
WRITE  . . . . . . . . . . . . .  	NUMBER	0040	
WRITE_PROTECT  . . . . . . . . .  	NUMBER	0000	

XA_CHAIN . . . . . . . . . . . .  	NUMBER	0084	
XDUP . . . . . . . . . . . . . .  	NUMBER	0045	
XDUP2  . . . . . . . . . . . . .  	NUMBER	0046	
XNAMETRANS . . . . . . . . . . .  	NUMBER	0060	

YEAR_MASK  . . . . . . . . . . .  	NUMBER	FE00	
YES  . . . . . . . . . . . . . .  	NUMBER	FFFF	
YES_BYTE . . . . . . . . . . . .  	V BYTE	0000	CONST	External
YES_FOUND  . . . . . . . . . . .  	NUMBER	0001	
YN_ARG . . . . . . . . . . . . .  	V WORD	0000	CONST	External

$$A_START_chkprmt  . . . . . . .  	L NEAR	0000	CODE	Global
$$A_STOP_chkprmt . . . . . . . .  	L NEAR	002C	CODE	Global
$$DO1  . . . . . . . . . . . . .  	L NEAR	0001	CODE
$$EN2  . . . . . . . . . . . . .  	L NEAR	0028	CODE
$$IF2  . . . . . . . . . . . . .  	L NEAR	0027	CODE
$$IF3  . . . . . . . . . . . . .  	L NEAR	0025	CODE
@CPU . . . . . . . . . . . . . .  	TEXT  0101h		
@FILENAME  . . . . . . . . . . .  	TEXT  chkprmt		
@VERSION . . . . . . . . . . . .  	TEXT  510		


    910 Source  Lines
    941 Total   Lines
    256 Symbols

  46518 + 250651 Bytes symbol space free

      0 Warning Errors
      0 Severe  Errors
